:4000000000080020110000006B0100006B01000010B500F057FE00F05BF900F0AFF8000010B572B69922154B12041A60EE22144B12021A602023C421124A89021360124A57
:40004000124C1160124A18201360D822114B12011A601223236000F0C9FD80220E4B52011A600E4A0E4B1A6000220E4B1A600E4B40321A601123236010BDC0460000024060
:400080000003024000000440080004403000104018000440080304400003014040FF008000000140280003400401014000000000000000000000000000000000000000004B
:4000C0000000000000000000000000000000000000000000000000000000000000000000000000000000000000000000000000000000000000000000000000000000000000
:4001000010B5064C2378002B07D1054B002B02D0044800E000BF0123237010BD1001002000000000FC100000084B10B5002B03D00749084800E000BF07480368002B00D106
:4001400010BD064B002BFBD09847F9E70000000014010020FC100000880000200000000010B562B600F0E0FAFEE710B500F084FF03680C2B00D1FEE7FEE70000F8B50025F0
:400180000F49104B01394A1C14D000221F685C689E68A018B24203D0B858A0500432F8E70200DE68141AA64201D020C2FAE710330139E8E700F066FFFFF7D2FFFEE7C046BC
:4001C0000100000034110000002370B50B480C4C0C4D9A002100032B00D8A95801338150202BF6D1FFF71CFF074B1A68002A00D11A608022054B92051A6070BD00000020EA
:400200006B010000000000008000002008ED00E0004700234118002A05D0013A881800781B18DBB2F7E7180070470000013810B50B2831D8C901494200F00AFF06090B0DAC
:400240000F111513171A1C21FF239B0113E0154B16E0154B0AE0154B12E0154B0BE0154B09E0154B02E0154B00E0154BC91814E0144B05E0144BC9180878C0B211E0134B15
:40028000C9180A7848788C780002230418430300C8781343000603E000210B7848780002184310BDC13F0000C53F0000C93F0000D03F0000D13F0000D63F0000D23F000032
:4002C000D43F0000D83F0000DC3F0000E03F00000C4B10B51A68102313400B4A00D113601368802B0DD10024022021001460FFF79DFFA04205D021000220FFF797FFFFF7F0
:4003000087FF10BD5400034080000020F8B5010006000320FFF78AFF040031000420FFF785FF0134E4012718002431000320FFF77DFF25000130C001B84209D203785A1EE8
:40034000D2B2FD2A00D80125E418E4B20130F3E731000120FFF76AFF6442E4B20623844203D16A4255416D422B401800F8BD0000F0B5BF4CA544019000F00AFA62B6019B8C
:40038000002B02D06B461B7901E0BA4B1B78DBB2039300250A23009502939621039B04AA49000AA800F0FCF9019B002B03D0029B013BDBB20293029B002B02D00028ECD1EC
:4003C00002E0002800D08BE004AB1988062900D849E11A7E0423012A52D104AA568BF21D8A4200D941E1962149008A4200D93CE10AAA92199279172A42D10022F3189BB2CB
:40040000002B09D0A0A99C48C91809180978013B521892B29BB2F3E70AAFBB19597952421B79090292B219430823914228D162E0342B00D0C8E0009B012B00D013E1032EF9
:4004400000D010E18022002155A800F04AFE80251F2155AB581904AB7519F21EC918ADB200F036FE832D00D0F7E004AB9D7F587F2D0205437F2D00D80EE1012300930933E6
:40048000002404AA548001210AAA5370230AD370002311709470221D92B2002A09D0A0A97548891809180978013A5B189BB292B2F3E7A0AA714912195B4251189BB20B7000
:4004C0006F491B0A51180B706E4B0734D2181723137004AAA1B27F3302320AA800F091F9019B002B00D158E7009B012B00D014E10123009351E77B783C79180031380A28E0
:400500002ED9614A1468002C26D0009A012A25D104AAD68007AE13710BAF0C2200213000069700F0DEFDB760310005A8A0472623B488FF339C4202D9B368BB4207D0B2687D
:40054000002A01D1002C04D13368DBB299E70E2396E70E23140094E7052392E705238FE700F080FD0B001900CFFF66FF3800CFFF3C004E0066FF5E006E00009B012B72D19A
:40058000002E70D13000FFF7C1FE43424341009C3B71330075E7009B012B64D1012E62D1002C60D1394B80211B681B689A0BD2B2002A01D19B04590E00237F2239717B719C
:4005C000BA71FB7104245CE7009B012B4BD1022E49D93DE7009B012B45D198E0009B012B41D12C337419FF339C423EDC55AB581932000BA900F06CFD0023A5B21C0040E7EF
:40060000002E30D107AB1900214A350011CA11C10BAA03CB03C2012308240093330030E7009B012B1FD1032E1DD104AA04AB977F5B7F3F021F430A237F2F00D920E748E055
:400640000020FFF763FE002802D18022114B1A6000F0A2F800F046FA05E001230025009302332C000DE704230AE7032308E7C0467CFDFFFF00110000A7FDFFFFACFDFFFFBC
:40068000ADFDFFFFAEFDFFFF2C0100208C0000200411000080000020224B1B681A68D3099BB2520601D001339BB2E0012D18A8B2834204D90123002500930933D1E755A906
:4006C00000F012F90028F5D10123050000930300C7E7E101C919C90180220020FFF799FD0600002C0DD17F2F0BD121000520FFF79DFD2100361A0620FFF798FDF6B2361A3E
:40070000F6B20AAB76421E7101240023B9E60025019BAB4200D0EBE63FE6A1239B009D44F0BDC0468C00002070B50020FFF7EEFD431E98410625144C4042236805401A685C
:40074000C021C03A0020FFF764FD63681B78181AC0B2834203D123681B68002B02D1002000F0BEF9094C2368402B01D0002D03D000202060FFF7FCFD1420FFF7F9FD80234B
:40078000236000F0AFF970BD8C0000208000002010B500F0C1FA10BD10B500F0CBFA10BDF8B504000F0016000120002C28D0002926D00A255D4300F0EBFA002810D000F04B
:4007C000E7FA0500AB2000F06DFA00F0E1FA8542F5D13900AF4200D929003180651807E00120013D00F08AF9002DE4D1102007E0AC4204D000F0B4FA20700134F8E7002069
:40080000F8BD70B501230C001500002805D0002903D000F001FB00232C80180070BD000082B06A460B4B0C4900930C4B01930C4B1A600C4A1160C0461A68120F0F2A04D047
:400840001A680020120F0A2A01D01868C0B202B07047C046B6E9000016000080300100200800104004001040094B0A4A0A491A600A4A1160C0461A68120F0F2A04D01A68AB
:400880000020120F0A2A01D01868C0B27047C04608001040B6E80000150000800400104082B06A460B4B0C4900930C4B01930C4B1A600C4A1160C0461A68120F0F2A04D00B
:4008C0001A680020120F0A2A01D01868C0B202B07047C046B6EA000017000080300100200800104004001040F0B50024A7B00294060003947F2854D8A14252D0802206A820
:4009000000F0E6FB294B04AF04937F23284D7B60284A294B2F601360C0462B6801921B0F0F2B03D02B681B0F0A2B01D02C68E4B20294029B002B36D100F0D7F90400FFF7DF
:400940006FFF0390039B002B02D1FFF78DFF0290029B002B16D1194A19490492049A0198360416430496124A2F600160C0462968090F0F2903D01168090F0A2901D0136842
:40098000DBB20293039B002B07D1FFF789FF0390039B002B01D0039B0293200000F0A9F901E004230293029827B0F0BDB6D70000080010400400104004000080B6D80000DE
:4009C0000500008010B5040000F08FF9102C04D803210C4A13688B430FE0202C05D80321084A13688B43023906E0302C06D80321044A13688B4301390B43136000F079F90C
:400A000010BDC046300010400B480C4A0C4B10B51B68116804680B4A9B00224002601C2213400A07920F1833D340074A9B181B78064ADBB2136010BD00000740280003407B
:400A4000080F0340FFFFFFBFCDF1FF0F0C0F0340024B18684000C00F7047C04600000740024B8000C31818681960704740000020F8B5032605003540B5400F00040006350B
:400A8000AE40AF4000F031F9A408054BA400E4182368B3431F43276000F02BF9F8BDC04600E400E01F2318401E3B8340014A13607047C04600E100E01F2318401E3B8340FE
:400AC000014A13607047C04680E100E01F2318401E3B8340014A13607047C04680E200E001BE7047034A044913689BB20B4313607047C0460CED00E00400FA0570B58025CB
:400B000004002D02064BAC4205D9586800F0E4F8044BE418F6E79868604300F0DDF870BD940000200080FFFFF0B585B000F0C4F8002846D000F0D9F80024234A234B0190D5
:400B40001B681068224A234D14602968224A9B001140A022520311431C2213400207920F1833D3401D4A1E4E53438022D2019B18DB0B013B0B432B60336830200393FFF73A
:400B800021FF8021174AC90513680B4313602A68154B1A40170001201034FFF7AFFFA3053B432B60F02CF6D10120FFF7A7FFFF23084A9B053B431360039B0198336000F08D
:400BC00098F805B0F0BDC04628000340080F03400C0F03400800074000F800C040420F003000104000000740FFFF3FC0F7B50500183D0400182D45D80126234B3700EB401B
:400C00009F433FD100F071F80190FFF721FF0097002802D0FFF7F8FE009607271B4E1C4A33681C49BB4333601B4BE3181B78DBB213601A4A1368BB431360194B0A68E3180C
:400C400018787F239A43034013430B60322000F043F8182C0ED033681C3CA408BB433C401C433460322000F037F83368AD08BB431D433560009B012B01D1FFF755FF019886
:400C800000F037F8F7BDC04611111101080F03400C0F0340180F0340CDF1FF0F100F0340B4F1FF0F10B5034B1B7B584300F014F810BDC04694000020014B1868C00F70470B
:400CC00000000740014A024B1A6070476588EDAC38000340000000000230800803D001300238FCD1C046C0467047EFF3108072B6704780F3108870478021064A10B5136817
:400D000009060B4313600820FFF7CCFE00F006F910BDC0460000094010B5054C2378002B03D100F085F801232370FFF7E5FF10BD4801002010B50820FFF7BEFE00F004F980
:400D4000054A082013685B005B0813600022034B1A60FFF7BBFE10BD00000940880F0940084B094A196813680020994208D013680133412B00D103000449C85C1360C0B207
:400D80007047C046E8010020E40100205C010020044B1868044B1A681B68904200D24130C01A7047E8010020E4010020134B144A30B515681C681900A54208D1114B1C68B9
:400DC0001F232340082B02D00F4B186015E013680133402B00D100230C68A342FCD002210A4CC0B221600A4CE0541360094B1A680A4202D11A680A431A6030BDA0010020FA
:400E0000580100200802094040020940800F0940A4010020880F094070B504004518AC4204D02078FFF7C2FF0134F8E770BD000070B50024072104251E4A1F4B08201A60F8
:400E40001E4B1F4A1C601F4B1A601F4B1F4A13601F4A11601F4A063914601F4A11601F4A13601F4B1C601F4B1D60FFF725FE03210820FFF7FDFD1C490820FFF7F1FD1B4B55
:400E80001C601B4B1C601B4B1C601B4B1C601B4B1D601B4B1C601A681A4B1A801A4B1C601A4B1C601A4B1C701A4B1C601A4B1C6070BDC0460B000002000009404000094043
:400EC00001000A00480009400700008000030940040309401003094044000940000209400402094050000940750F0000880E0940C80E0940480F0940080F0940C80F094075
:400F0000880F094050010020E8010020E40100205401002058010020A0010020064A074B11680B40902109040B431360044B1A88044B1A607047C04600000240FFFF0FFFF9
:400F400050010020880F0940064A074B11680B401360064B1A68E423DB001340044A13807047C04600000240FFFF0FFF880F094050010020254B70B51B68002B00D0984710
:400F8000234B1B685B071CD520241F2021490B680133412B00D100231F4A15681F4AAB4203D113681E4B1C7004E012681D4DD2B2EA540B601C4B1B680342E8D104221B4B10
:400FC0001A601B4B1B689B071FD51F20194C1A4A21681368994210D013680133402B00D100231649164DC95CC9B229601360154B1B680340082BEBD104E00221124A1368D2
:401000008B4313600222114B1A6070BD4C010020CC0F0940E8010020E401002040030940540100205C01002008030940C00F09408C0F094058010020A0010020A4010020DC
:401040004002094008020940880F0940800F094002B4714649084900095C49008E4402BC7047C04603B47146490840004900095E49008E4403BC7047014B18687047C0460F
:40108000080100200E4B70B500251E000D4CE41AA410A54204D0AB00F35898470135F8E700F036F8084B00251E00084CE41AA410A54204D0AB00F35898470135F8E770BD0A
:4010C0001C1100001C1100001C11000024110000002310B59A4203D0CC5CC4540133F9E710BD03008218934202D019700133FAE7704700000012000092000000000000003F
:40110000FF000000A9110319003C010143000000F8B5C046F8BC08BC9E46704729010000C9010000F8B5C046F8BC08BC9E467047010100004811000088000020880000004E
:40114000E00000000000000000000000F4100000F8100000010000000000E02EC05D00001800000000366E010000000000000000000000000000000000000000000000009A
:4011800000000000000000000C1100000000000000000000000000000000000000000000000000000000000000000000000000000000000000000000000000000000000012
:4011C0000000000000000000A80000200000000000000000000000000000000000000000000000000000000000000000000000000000000000000000000000000000000027
:4012000000000000000000000000000000000000000000000000000000000000000000000000000000000000000000000000000000000000000000000000000000000000AE
:40124000000000000000000000000000000000000000000000000000000000000000000000000000000000000000000000000000000000000000000000000000000000006E
:40128000000000000000000000000000000000000000000000000000000000000000000000000000000000000000000000000000000000000000000000000000000000002E
:4012C00000000000000000000000000000000000000000000000000000000000000000000000000000000000000000000000000000000000000000000000000000000000EE
:403FC00000000000000000000000000000000000000000000100000000000000000000000000000000000000000000000000000000000000000000000000000000000000C0
:0200000490303A
:020000006B7F14
:0200000490402A
:1000000000000000000000000000000000000000F0
:0200000490501A
:0C0000000002190311A9000119087D2855
:0200000490600A
:0100000001FE
:00000001FF
